:020000040800F2
:1000000000100020A90B0008F90B0008F90B0008EC
:1000100000000000000000000000000000000000E0
:10002000000000000000000000000000F90B0008C4
:100030000000000000000000F90B0008C1090008E2
:10004000F90B0008F90B0008F90B0008F90B000880
:10005000F90B0008F90B0008F90B0008F90B000870
:10006000F90B0008A50E0008D5100008F90B0008D0
:10007000F90B0008F90B0008F90B0008F90B000850
:10008000F90B0008F90B0008F90B0008F90B000840
:10009000F90B0008F90B0008F90B0008F90B000830
:1000A000F90B0008F90B0008F90B00081110000803
:1000B000F90B0008F90B0008F90B0008F90B000810
:1000C00090B583B000AF02003960FB1D1A70FB1DB4
:1000D0001B787F2B32D92F4AFB1D1B7819000F2369
:1000E0000B40083B9B0806339B00D31804331B6866
:1000F000FA1D1278110003220A40D200FF2191401C
:100100000A00D2431A4011003B689B01FF221A40AB
:10011000FB1D1B78180003230340DB009A401D4899
:10012000FB1D1B781C000F232340083B9B080A4340
:1001300006339B00C31804331A6027E0164AFB1DE0
:100140001B785BB29B08C0339B009B58FA1D12784A
:10015000110003220A40D200FF2191400A00D2433D
:100160001A4011003B689B01FF221A40FB1D1B78BF
:10017000180003230340DB009A400748FB1D1B784F
:100180005BB29B080A43C0339B001A50C046BD4671
:1001900003B090BD00ED00E000E100E080B582B06A
:1001A00000AF78607B685A1E80235B049A4201D3BB
:1001B000012310E00A4B7A68013A5A6001235B423E
:1001C00003211800FFF77CFF054B00229A60044BC7
:1001D00007221A6000231800BD4602B080BDC04649
:1001E00010E000E080B582B000AF7860064B0022DE
:1001F0001A60C046044B1B687A689A42FAD8C04617
:10020000C046BD4602B080BD08000020B0B5B4B005
:1002100000AF0023CC243A1913600023C822BA1877
:1002200013603B1D180080231A00002101F098F88C
:10023000C723FB1800221A70C623FB1800221A706D
:10024000C423FB1800221A700023BC22BA181360C2
:10025000BB23FB1801221A70D54B5A69D44BC0211D
:10026000C9020A435A61D24BDA69D14B8121490054
:100270000A43DA619023DB051A689023DB05CD4938
:100280000A431A609023DB05DA689023DB05CA492C
:100290000A43DA609023DB051A6A9023DB05882184
:1002A00049050A431A62C54B1A68C44B08210A4320
:1002B0001A60C24AC14B126A1A62C14BC14ADA6261
:1002C000BF4B00225A62BE4B00225A60BC4B012237
:1002D0009A60BB4BBC4A9A61B94B22221A62B84B56
:1002E00000229A62B64B01221A60B84BFF22DA62F2
:1002F000B64B00225A62B54B00225A63B34B0A2216
:100300009A62B24B68229A61B04B01221A62AF4BDB
:1003100000225A60AD4B01221A6040233A19136043
:10032000C323FB1800221A7000F080FC002000F0AC
:10033000E7FDA74B1800FFF731FFC523FB1800228C
:100340001A7000F0E3FC0200A24B1A60CC23FB18E9
:100350001A68C823FB181B689A4204D1C623FB18ED
:100360001B78002B03D0C523FB1801221A70C4216F
:100370007B181B78002B08D0964B1B68964A93423B
:1003800010DC7B1800221A700CE0924B1968C42311
:10039000FB180122101CAF229200914201DC0022C6
:1003A000101C1870C423FB181B78002B0ED0CC2215
:1003B000BB181B68022B09D9C323FB181B78072B1A
:1003C00004D8BB181B68013BBA18136000F0A4FEE8
:1003D000031E13D0C322BB181B78072B0AD8CC23CB
:1003E000FB181B68BC2179180B60BB23FB18BA18DB
:1003F00012781A70C323FB1809221A70C723FB183E
:1004000000221A70C323FB181B780A2B00D9FCE1C9
:100410009A00724BD3181B689F460023B422BA1867
:1004200013601AE0CC217B181B681A067B181B6826
:100430001B04D2187B181B681B02D2187B181B6880
:10044000D1183B1DB4203A1812689200D150020016
:10045000BB181B680133BA181360B423FB181B6860
:100460001F2BDFD9C723FB18CC22BA1812681A70C9
:10047000E6E10023B022BA1813600FE0CC23FB188A
:100480001B6819043B1DB0203A1812689200D15025
:100490000200BB181B680133BA181360B023FB18A5
:1004A0001B681F2BEAD9CBE10023AC22BA181360DA
:1004B0000FE0CC23FB181B6819063B1DAC203A1833
:1004C00012689200D1500200BB181B680133BA18A1
:1004D0001360AC23FB181B681F2BEAD9B0E1002383
:1004E000A822BA1813600FE0CC23FB181B6819026E
:1004F0003B1DA8203A1812689200D1500200BB1888
:100500001B680133BA181360A823FB181B681F2B44
:10051000EAD995E10023A422BA1813600CE03B1D30
:10052000A4203A18126892000021D1500200BB1892
:100530001B680133BA181360A423FB181B681F2B18
:10054000EDD9C723FB18CC22BA1812681A7077E1CC
:100550000023A022BA1813601EE0A0217B181B689C
:10056000DB001A00CC23FB181B68934207D93B1D04
:100570007A181268920001214942D15006E03B1DD1
:10058000A022BA18126892000021D150A022BB18F4
:100590001B680133BA181360A023FB181B681F2BBC
:1005A000DBD94DE100239C22BA18136048E0C04615
:1005B0000010024040A0000001500000000400486C
:1005C00000040040FFFF0000010200000020004086
:1005D00000350C000400002025020000081400086B
:1005E000CC257B191B680721180000F0FBFD0300D8
:1005F0001A009C243B191B689A4214D97B191B686A
:100600000721180000F0EEFD03001A003B191B68DB
:1006100007339A4207D23B1D3A1912689200012112
:100620004942D15006E03B1D9C22BA181268920044
:100630000021D1509C22BB181B680133BA181360EB
:100640009C23FB181B681F2BCAD9F9E000239822B2
:10065000BA1813603BE09823FB181B6803211800AD
:1006600000F006FE03001A00CC23FB181B68D31809
:100670000321180000F0F2FD0B00022B17D01FD849
:10068000002B02D0012B09D01AE03B1D9822BA188A
:1006900012689200FF210904D15012E03B1D9822FC
:1006A000BA1812689200FF210906D15009E03B1DDB
:1006B0009822BA1812689200FF210902D15000E076
:1006C000C0469822BB181B680133BA1813609823E0
:1006D000FB181B681F2BBED9B2E0C523FB180022F4
:1006E0001A7000F02FFD031E65D0C423FB181B7881
:1006F00001225340DBB2002B5DD000F081FC0300EF
:1007000084217A181360C323FB180A221A707B18FD
:100710001B681B78002B00D08FE000239422BA18AE
:10072000136035E094203B181B689B00043384243D
:100730003A191268D3181B7819003B181B689B00E4
:1007400003333A191268D3181B781B020A001A43A4
:100750003B181B689B00013319003B191B685B1891
:100760001B781B041A433B181B689B000233391982
:100770000968CB181B781B06134319003B1D3A1858
:1007800012689200D1503B181B6801333A1813606D
:100790009423FB181B681F2BC4D98423FB181B68E8
:1007A00081331A00C723FB1812781A70C523FB186F
:1007B00001221A7043E0C423FB181B78002B3ED0A3
:1007C000C523FB1801221A7000239022BA18136067
:1007D0000CE03B1D90203A18126892000021D15085
:1007E0000200BB181B680133BA1813609023FB1872
:1007F0001B681F2BEDD9C723FB1800221A701EE0BF
:10080000C523FB1800221A701AE000238C22BA18A4
:1008100013600CE03B1D8C203A18126892000021F6
:10082000D1500200BB181B680133BA1813608C2327
:10083000FB181B681F2BEDD902E0C04600E0C04644
:10084000C423FB181B78002B0ED0C523FB180122F4
:100850001A70574B1B78DBB2002B02D0FF231A040F
:1008600000E000223B1D1A60C523FB181B78002BFB
:1008700026D0504BC722BA1812785A630023882218
:10088000BA18136011E072B6C0463B1D88243A19AD
:1008900012689200D358180000F070FC62B6C0468F
:1008A0003B191B6801333A1913608823FB181B6836
:1008B0001F2BE8D9CC23FB181B68C822BA18136079
:1008C000C322BB181B780A2B03D0BB181B78092B3B
:1008D00004D1C423FB181B78002B02D00520FFF79E
:1008E00081FC354B5B6A1AB2CC217B181B681BB2AA
:1008F0009A4203DD00237A18136019E0CC217B189B
:100900001B681BB21A002C4B5B6A1BB2D31AFF2B5D
:1009100003DDFF237A1813600AE0CC217B181B68E3
:100920001BB21A00244B5B6A1BB2D31A7A181360ED
:10093000214B00225A62C6217B181B78002B0AD05B
:100940009023DB051B690122134000D1F5E47B18DD
:1009500000221A70F1E49023DB051B690122134089
:1009600000D0EAE4C623FB1801221A70C322BB1888
:100970001B78082B0BD9BB18BB22BA1812781A7037
:10098000BC23FB181B68CC22BA181360D5E4C32320
:10099000FB181B780133094A134004D5013B082298
:1009A0005242134301331A00C323FB181A70C4E4E4
:1009B0000C000020002000400004004007000080E0
:1009C00080B500AF114B1B685A1E104B1A600F4BBD
:1009D0001B68002B11D10D4B0A221A600C4B1B789F
:1009E000DBB25A1E9341DBB201225340DBB21A1C28
:1009F00001231340DAB2064B1A70064B1B685A1CCF
:100A0000044B1A60C046BD4680BDC04600000020B1
:100A10000C0000200800002080B500AF1A4B1A68B7
:100A2000194B01210A431A60174B5A68164B174994
:100A30000A405A60144B1A68134B15490A401A6051
:100A4000114B1A68104B13490A401A600E4B5A6832
:100A50000D4B11490A405A600B4BDA6A0A4B0F21C1
:100A60008A43DA62084B1A6B074B0C490A401A6337
:100A7000054B5A6B044B01218A435A63024B0022F7
:100A80009A60C046BD4680BD001002400CB8FF0809
:100A9000FFFFF6FEFFFFFBFFFFFFC0FFECFEFFFFC7
:100AA00080B582B000AF224B5A68214B80214902A9
:100AB0000A435A601E4B0122DA621D4B1A681C4B16
:100AC000802149020A431A60C046194B1A688023E4
:100AD0009B021340F9D0164B5A68154BA02189038D
:100AE0000A435A60124B1A68114B802149040A4389
:100AF0001A60C0460E4B1A6880239B041340F9D03D
:100B00000B4B5B687B607B68032293437B607B6855
:100B1000022213437B60064B7A685A60044B1A68C2
:100B2000034B01218A431A60C046BD4602B080BD16
:100B30000010024080B500AFFFF76EFFFFF7B0FF77
:100B4000C046BD4680BDC04680B586B000AFF860E7
:100B5000B9607A60BB683B61FB687B6107E07A69DA
:100B6000131D7B613B69191D396112681A603A696E
:100B70007B689A42F3D3C046C046BD4606B080BDEE
:100B800080B582B000AF7860396004E07B681A1DE0
:100B90007A6000221A607A683B689A42F6D3C046AF
:100BA000C046BD4602B080BD80B500AF0B4A0C49BF
:100BB0000C4B1800FFF7C8FF0B4A0C4B1100180034
:100BC000FFF7DEFF0A4A0B4B11001800FFF7D8FFB2
:100BD000FFF7B0FFFFF71AFBC046FDE70400002057
:100BE000000000203414000844020020040000200B
:100BF000440400204402002080B500AFC046FDE759
:100C000080B582B000AF0200FB1D1A70FB1D1B787F
:100C10001A001F231A40044B012191400A001A6058
:100C2000C046BD4602B080BD00E100E080B500AF27
:100C3000254B5A69244B01210A435A61224B9A6978
:100C4000214B802189000A439A61204B1A681F4B6F
:100C50001F490A401A601F4B10225A601D4B1E4A42
:100C60009A601C4B1D4ADA601A4B1D4A1A60092013
:100C7000FFF7C6FF1B4B802212069A60C046194B35
:100C80009B68002BFBDB174B1B6C164B00229A60FA
:100C9000144B154ADA60134B802212061A61114B6D
:100CA00007225A61114B1A68104BC02109040A43EC
:100CB0001A600C4BC02292029A620A4B05229A607B
:100CC000C046BD4680BDC046001002400000014045
:100CD000FFE0FFFF08000240402401401000002018
:100CE000A325000000240140032000000827014044
:100CF00080B582B000AF044B7B607B681B889BB2E1
:100D00001800BD4602B080BDB8F7FF1F80B582B0A5
:100D100000AF164B7B60164B1B68002B00DA0F33BD
:100D20001B111A00134B1B6853431349180000F0A2
:100D30009FFA03001B013B60FFF7DAFF03009A02F2
:100D40003B68D31A3B603A6813009B009B185B001A
:100D50007968180000F08CFA03002D33FF333B60F4
:100D60003B681800BD4602B080BDC0465815000063
:100D70003400002030000020330D000080B582B028
:100D800000AF044B7B607B681B889BB21800BD469C
:100D900002B080BDBAF7FF1FB0B58AB000AF002324
:100DA0003B620023FB61FFF7E9FF0300BB61002307
:100DB0007B6217E07B6A5A00354B5200D35A9BB2D4
:100DC0001A003B6A9B183B627B6A5B005A1C304BE3
:100DD0005200D35A9BB21A00FB699B18FB617B6AD5
:100DE00001337B627B6A072BE4DDFB69DB08FB6177
:100DF0003B6ADB083B62BB69264A5343F96918002A
:100E000000F0F0F903007B613B6A9B023B61224BDF
:100E10001A6813009B009B189A009B185B0119002D
:100E20007A691300DB009B1A5B01CB189A121A4BEC
:100E30001A601A4B1B68BB60DB17FB60C82292006C
:100E40000023B868F96800F069FA02000B0010008E
:100E500019003A691300DB009B1A5B013B60DB174A
:100E60007B603A687B6812184B41002B03DA0C4810
:100E7000002112184B419905940A0C439D1222003F
:100E80002B00064B1A60C046BD460AB0B0BDC04636
:100E900010000020330D000030000020340000203E
:100EA000FF03000080B582B000AF094B1B687B6078
:100EB000074B7A680F210A405A607B680222134070
:100EC00001D0FFF769FFC046BD4602B080BDC046F5
:100ED0000000024080B582B000AF0200FB1D1A7016
:100EE000FB1D1B781A001F231A40044B012191405F
:100EF0000A001A60C046BD4602B080BD00E100E0B5
:100F000080B584B000AF78600023FB60324BBB60DB
:100F100008E0BB6800221A70FB680133FB60BB6805
:100F20000133BB60FB68802BF3D92C4B7A681A60C5
:100F30002B4B00221A702B4B5A692A4B2A490A4321
:100F40005A61284B9A69274B8021C9010A439A614B
:100F50009023DB051A689023DB058021C9000A4332
:100F60001A609023DB059A6A9023DB0520210A434F
:100F70009A629023DB051A689023DB0580218903A0
:100F80000A431A609023DB055A6A9023DB0580210F
:100F900049000A435A62154BC022DA60134B012202
:100FA0009A60124B802292015A60104B25221A60DF
:100FB0000F4B1A680E4B0F490A401A600E4B0F4A2E
:100FC0001A600A20FFF786FF1B20FFF783FFC04649
:100FD000BD4604B080BDC04640000020380000205F
:100FE0003D000020001002400100020000380140D6
:100FF00000000140FFFBFFFF3000024082200000A4
:1010000080B500AF014B1800BD4680BD40000020F8
:1010100080B582B000AF284BDB697B60264B0E2287
:101020001A627B680222134033D0234B9A68224B0A
:1010300040218A439A60204B08229A611F4B1A680C
:101040001E4B01218A431A60C0461C4B1B680122BB
:101050001340FAD1194B1A4ADA60184B194A9A60B0
:10106000164B194A5A60154B1A68144B01210A4352
:101070001A60114B08229A610F4B9A680E4B40215F
:101080000A439A60114B01221A70114B01221A7007
:101090000BE07B682022134007D00D4B1B78DBB29E
:1010A000012B02D0044B08229A61BFF34F8FC04638
:1010B000C046BD4602B080BD00380140300002404D
:1010C0004000002024380140010200003D000020C3
:1010D0003C00002080B582B000AF0D4B1B687B60E8
:1010E0000B4B7968F02212010A405A607A6880231B
:1010F0009B00134004D0064B1B68064B00221A705D
:10110000BFF34F8FC046C046BD4602B080BDC0464B
:10111000000002403C00002080B582B000AF72B6F3
:10112000C046FB1D064A12781A70054B00221A7041
:1011300062B6C046FB1D1B781800BD4602B080BDDC
:101140003D00002080B582B000AF094B5B68094AC2
:10115000D31A7B60084B1B6881337A689A4201D9A5
:10116000012300E000231800BD4602B080BDC04648
:1011700030000240010200003800002000B570B4C9
:101180001049114A114B124C124D28420ED004D175
:101190004000013CF9D170BC00BD0A600E4E00F069
:1011A0000EF80B600D4E00F00AF8F1E70A600C4EE5
:1011B00000F005F80B60084E00F001F8E8E7013E8A
:1011C000FDD170471800004808000000000008002A
:1011D0002000000000000080050000000200000068
:1011E00001000000002934D00123002210B48842FD
:1011F0002CD301242407A14204D2814202D2090146
:101200001B01F8E7E400A14204D2814202D2490066
:101210005B00F8E7884201D3401A1A434C08A04209
:1012200002D3001B5C0822438C08A04202D3001B9F
:101230009C082243CC08A04202D3001BDC082243B6
:10124000002803D01B0901D00909E3E7100010BCF6
:10125000704701B5002000F05FF802BD0029F8D00A
:1012600003B5FFF7C1FF0EBC4243891A1847C046B9
:10127000002941D010B404004C40A44601230022B0
:10128000002900D54942002800D5404288422CD38D
:1012900001242407A14204D2814202D209011B0188
:1012A000F8E7E400A14204D2814202D249005B0087
:1012B000F8E7884201D3401A1A434C08A04202D3EF
:1012C000001B5C0822438C08A04202D3001B9C0830
:1012D0002243CC08A04202D3001BDC082243002892
:1012E00003D01B0901D00909E3E710006446002C74
:1012F00000D5404210BC704701B5002000F00CF84A
:1013000002BDC0460029F7D003B5FFF7B3FF0EBCFE
:101310004243891A1847C0467047C046F7B5040CC7
:101320000D0091B20F0061438C460600019383B219
:10133000100C5F43444358433B0C60441B189942D4
:1013400002D9802149026418019955437143180C50
:1013500004191B04BFB24919D819091903B0F0BD0B
:10136000F0B50500830749D0541E002A45D003007C
:101370000326CAB202E00135013C3ED301332A7094
:101380003342F8D1032C30D9FF250D402A022A43DD
:10139000150415430F2C34D92700103F3F093E0197
:1013A000B4461E001A0010366644156055609560FC
:1013B000D5601032B242F8D101373F01DB190F2757
:1013C0000C22274022403C00002A0ED03E1FB608C7
:1013D000B400A4461A001C1D644420C2A242FCD1E1
:1013E00003240136B6009B193C40002C05D0C9B23D
:1013F0001C19197001339C42FBD1F0BD030014008D
:10140000C0E72700E2E7C0461405000872040008A0
:10141000A8040008DE0400081A04000850050008AB
:10142000A40500084C0600080A080008DA060008AF
:0414300000080008A8
:041434000A000000AA
:0400000508000BA93B
:00000001FF
